:1000000025C049C048C047C046C0D2C044C043C054
:1000100042C041C040C03FC03EC03DC03CC00000E7
:100020000000370000000000380002020202020255
:10003000020202020102040810202004100801023A
:1000400000000400000000002703810311241FBEEC
:10005000CFE5D2E0DEBFCDBF10E0A0E6B0E0E0EC3F
:10006000F9E002C005900D92A039B107D9F720E060
:10007000A0E9B0E001C01D92A23BB207E1F710E099
:10008000C5E2D0E003C02197FE0163D3C432D1079B
:10009000D1F7D8D089C4B4CF90E0FC01E25CFF4F27
:1000A0002491FC01EC5CFF4F3491FC01E65DFF4FB5
:1000B000E491EE23B1F0222329F02230F9F090F4FC
:1000C0002130C1F0F0E0EE0FFF1FEC5DFF4FA59176
:1000D000B4918FB7F8949C91E32FE095E923EC93CA
:1000E0008FBF0895233011F0243061F78CB58F7DD8
:1000F0008CBDE8CF8AB58F778ABDE4CF8AB58F7D76
:10010000FBCFCF93DF9390E0FC01EC5CFF4F249199
:10011000865D9F4FFC0184918823D1F090E0880F89
:10012000991FFC01E25EFF4FA591B491FC01EC5DCB
:10013000FF4FC591D49161110EC09FB7F8948C9177
:10014000E22FE0958E238C932881E223E8839FBFE2
:10015000DF91CF9108958FB7F894EC91E22BEC9357
:100160008FBFF6CF3FB7F89480919500909196009D
:10017000A0919700B091980022B708B601FE05C083
:100180002F3F19F00196A11DB11D3FBFBA2FA92F16
:10019000982F8827BC01CD01620F711D811D911D13
:1001A00043E0660F771F881F991F4A95D1F708957E
:1001B0001F920F920FB60F9211242F933F938F939C
:1001C0009F93AF93BF938091910090919200A091E3
:1001D0009300B09194003091900026E0230F2D37CA
:1001E00058F50296A11DB11D2093900080939100B7
:1001F00090939200A0939300B09394008091950007
:1002000090919600A0919700B09198000196A11D41
:10021000B11D8093950090939600A0939700B093A2
:100220009800BF91AF919F918F913F912F910F9027
:100230000FBE0F901F90189529E8230F0396A11D5C
:10024000B11DD2CFCF93DF93CDB7DEB7EA970FB60C
:10025000F894DEBF0FBECDBF78948AB582608ABDA8
:100260008AB581608ABD83B7826083BF83B78160AE
:1002700083BF89B7826089BF80B7826080BF80B743
:10028000816080BF329A319A3098379A8CB58064F9
:100290008CBD80919E0090919F0097FD05C061E00C
:1002A00030DF80919E00F8DE81E0809399009E010E
:1002B000255D3F4F3BAB2AAB87E0E6E6F0E0DE0191
:1002C000949601900D928A95E1F787E0EDE6F0E0D3
:1002D000DE015D9601900D928A95E1F787E0E4E7F3
:1002E000F0E0DE01569601900D928A95E1F787E0E5
:1002F000EBE7F0E0DE011F9601900D928A95E1F7A1
:1003000087E0E2E8F0E0DE01189601900D928A9510
:10031000E1F787E0E9E8F0E0DE01119601900D9247
:100320008A95E1F77E0134E2E30EF11C3E014FE0D5
:10033000640E711CCE014D9699AF88AFFE013896C0
:10034000FFABEEAB9E012A5E3F4F3DAB2CABAE0147
:100350004F5F5F4F6A0110E000E0F3016081802F82
:10036000DED1F7012081280FEEA9FFA96081802F3F
:10037000D6D1E8ADF9AD8080880D90E0B0E0A0E086
:10038000BA2FA92F982F88274C015D01A22AF601C8
:100390006081802FC4D1ECA9FDA99081890FA501AE
:1003A0009401282BDA01C9011D0144245524B22CE3
:1003B000492F5A2F6B2F7727A42E8AAF4101242E65
:1003C000312C482E512C30E020E080919A00909101
:1003D0009B0028173907A8F5E091A0004AADD50188
:1003E000EE2369F0F0E0C401BF01A2D1B92FCF0123
:1003F000B1019ED1A92FCF01B2019AD1492F5091BD
:10040000A600E091A100F091A2008091A3005813F2
:1004100012C1C90163E070E08BD18E0F9F1FE09184
:10042000A300E80FF92FF11DB083E091A400E80FBD
:10043000F92FF11DA0835091A500850F911DFC019E
:1004400040832F5F3F4F2D32310509F0BECF8091A1
:10045000A1009091A200892B09F49DC083DE8090B9
:10046000A7009090A800A090A900B090AA006815DD
:1004700079058A059B0540F46093A7007093A80056
:100480008093A9009093AA008090A7009090A80064
:10049000A090A900B090AA00681979098A099B095F
:1004A0006C32714081059105C8F2F89480919C00EE
:1004B00090919D009CA78BA7A091A100B091A20054
:1004C000FD0131968C9189AB1DA698B38091AD004A
:1004D000982B98AB98B3809589238FA78FA58EA76B
:1004E00089A987FF02C088A98EA758A96FA549A925
:1004F0003EA52DA58BA59CA558BB262F38BB00C0BB
:1005000046FD252F68BB00C058BB362F28BB00C056
:1005100045FD352F68BB00C058BB262F38BB00C037
:1005200044FD252F68BB00C058BB362F28BB00C038
:1005300043FD352F68BB00C058BB262F38BB00C019
:1005400042FD252F68BB00C058BB362F28BB00C01A
:1005500041FD352F68BB00C058BB262F38BB00C0FB
:1005600040FD252F68BB019758BB362F28BB419112
:1005700047FD352F68BB01F649AB3EA72DA79CA7C9
:100580008BA77894EFDD6093A7007093A800809309
:10059000A9009093AA00E6DD1B012C0184E6882EB9
:1005A000912CA12CB12CDEDD621973098409950907
:1005B000683E734081059105B0F321E0821A9108ED
:1005C000A108B10838EE230E33E0331E411C511C44
:1005D00081149104A104B10431F70F5F1F4F01157D
:1005E00051E0150709F0B9CE8FEFE81AF80A9FEF2E
:1005F000691A790AE8ADF9AD3196F9AFE8AF2EA9DD
:100600003FA92F5F3F4F3FAB2EAB4CA95DA94F5F7A
:100610005F4F5DAB4CAB5FEFC51AD50A8AA99BA9AA
:100620008E159F0509F097CEE0E0F0E0EF2B09F47E
:1006300043CEE6DC41CEC901880F991F880F991F70
:100640008E0F9F1FFC01E50FF11D1082E8CE109266
:1006500099001092A0001092A7001092A80010928A
:10066000A9001092AA0081E08093A6008093A300C5
:100670001092A40082E08093A50087E890E0909318
:100680009D0080939C006BD09093A2008093A1006A
:10069000009771F127E8FC0111922A95E9F78DE2A4
:1006A00090E090939B0080939A0082E090E090937A
:1006B0009F0080939E0080919900882329F061E03B
:1006C00082E01FDD82E0E8DCECE2F0E0E491F0E0C3
:1006D000EE0FFF1FEC5DFF4F859194919093AC005E
:1006E0008093AB00E6E3F0E0E491E093AD00089581
:1006F00010929D0010929C0010929B0010929A0004
:10070000D4CF8091A1009091A200C5D080919E008D
:1007100090919F0097FD02C060E0F3CC0895002403
:1007200080FD060E660F11F08695D1F7802D089595
:100730000024552704C0080E591F880F991F0097E1
:1007400029F076956795B8F37105B9F7802D952F47
:100750000895EE0FFF1F0590F491E02D09940F937B
:100760001F93CF93DF938230910510F482E090E0E5
:10077000E091B000F091B10030E020E0B0E0A0E006
:10078000309799F42115310509F44AC0281B390B1B
:1007900024303105D8F58A819B816115710589F175
:1007A000FB0193838283FE0111C04081518102814C
:1007B000138148175907E0F04817590799F4109723
:1007C00061F012960C93129713961C933296CF01F8
:1007D000DF91CF911F910F9108950093B000109376
:1007E000B100F4CF2115310551F04217530738F00D
:1007F000A901DB019A01BD01DF01F801C1CFEF01C1
:10080000F9CF9093B1008093B000CDCFFE01E20FFD
:10081000F31F819391932250310939832883D7CFD5
:100820002091AE003091AF00232B41F42091620063
:10083000309163003093AF002093AE0020916000B0
:10084000309161002115310541F42DB73EB740913B
:10085000640050916500241B350BE091AE00F091CF
:10086000AF00E217F307A0F42E1B3F0B2817390740
:1008700078F0AC014E5F5F4F2417350748F04E0FFC
:100880005F1F5093AF004093AE00819391939FCF31
:10089000F0E0E0E09CCFCF93DF930097E9F0FC011C
:1008A000329713821282A091B000B091B100ED0195
:1008B00030E020E01097A1F420813181820F931F56
:1008C0002091AE003091AF002817390709F061C0C0
:1008D000F093AF00E093AE00DF91CF910895EA016D
:1008E000CE17DF07E8F54A815B819E01411551056E
:1008F000B1F7E901FB83EA8349915991C40FD51FF0
:10090000EC17FD0761F4808191810296840F951F99
:10091000E90199838883828193819B838A83F0E0B4
:10092000E0E012968D919C9113970097B9F52D9167
:100930003C911197CD010296820F931F2091AE003A
:100940003091AF002817390739F6309751F51092DA
:10095000B1001092B000B093AF00A093AE00BCCF36
:10096000D383C28340815181840F951FC817D90753
:1009700061F44E5F5F4F88819981480F591F518301
:1009800040838A819B81938382832115310509F0FD
:10099000B0CFF093B100E093B0009ECFFD01DC0139
:1009A000C0CF13821282D7CF10E0C5E2D0E003C0DF
:1009B000FE01CFDE2196C632D107D1F7F894FFCFE2
:1009C0000000B2008000FFFF000000FFFF00FFFFFB
:1009D000FF0000FF000000FFFFFFFF00FF0000011D
:1009E0000000010000FF0001FF000001000000FF07
:00000001FF
